:100000000C946C060C94A4060C94A4060C94A40600
:100010000C94A4060C94A4060C94A4060C94A406B8
:100020000C94A4060C94A4060C9413280C94E528B4
:100030000C9434220C94A4060C94A4060C94A406EC
:100040000C94A4060C94A4060C94A4060C94A40688
:100050000C94A4060C94BC220C94A4060C94A40644
:100060000C94A4060C94A4060C94A4060C94A40668
:100070000C94A4060C94A4060C94A4060C94A40658
:100080000C94A4060C94A4060C94A4060C94A40648
:100090000C9483080C94A4060C94A4060C94A40657
:1000A0000C94A4060C94A4060C94A406960B960B30
:1000B000C20BC20B2A0C480C600D600D530CEC0CEB
:1000C000FD0CFD0C611E4F1E681EDA1D151F151F4D
:1000D0004C1E151F151F951E151FA91EF51E151F59
:1000E000151F151F151FC91E151F151FC61E151F0D
:1000F000811E151F151F0F1F0F1F0F1F0F1F0F1F13
:100100000F1F0F1F0F1F0F1F111F151F611E441EF2
:10011000151F151F151F151F151F151F151F151F3F
:10012000151F151F111F151F151F4C1E151F0D1F05
:100130000D1F0D1F0D1F0D1F0D1F0D1F0D1F0D1F5F
:10014000111F52297929712A7929712AC529E8298B
:10015000712A3F2A4E2A253032583A20253031362E
:100160006225730A00722F63203031323334353602
:100170003738394142434445460A005000E400E61E
:10018000000000510063004F0062001B00E30035D7
:100190000019000000290010002C00015137000058
:1001A000000000590058005A005B001D00E200E00A
:1001B0000006000E00000011000500340038003673
:1001C0000000005C0057005D005E0007000400E1D5
:1001D0000009000D003A000B000A00E50033000F93
:1001E000003000520000000000000016001400392A
:1001F0000015000C003C0018001700000000000073
:1002000000000000000000000000000000000000EE
:1002100000000000000000000000002E002D00275C
:1002200000310053002A005400550020001F000038
:1002300000210026003B00240023002F00130012A1
:100240000028005F005600600061001A001E002BAD
:1002500000080025003D001C00220044004300422D
:100260000045004C004E0049004B0000000000001B
:1002700000000041003E0040003F004A00650001D0
:100280000000004E0001004D0001000100010001CE
:100290000001000000010001000100010001000058
:1002A0000000000100010001000100010001000147
:1002B0000001000100000001000100010001000137
:1002C0000000000100010001000100010001000127
:1002D0000001000100010001000100010001000116
:1002E0000001004B000000000000000100010001BF
:1002F00000010046000100010001000000000000B4
:1003000000000000000000000000000000000000ED
:1003100000000000000000000000000100010001DA
:1003200000010001000100010001000100010000C6
:100330000001000100010001000100010048004728
:1003400000010001000100010001000100010001A5
:100350000001000100010001000100010001000195
:1003600000010001004D0001004A000000000000F3
:100370000000000100010001000100444542554712
:100380003A2064697361626C65642E0A00444542D8
:1003900055473A20656E61626C65642E0A000A005A
:1003A00025303258006C65645F7461736B3A2000CD
:1003B0004F6E6573686F743A206163746976653A4D
:1003C0002025640A00290A002575002F00257500E4
:1003D0005D280025640020002564002000256400BD
:1003E00020002564007C0025303258006D6F757345
:1003F000656B6579205B62746E7C7820792076204D
:10040000685D287265702F61636C293A205B00314A
:100410003A0964656C6179282A31306D73293A2074
:1004200025750A323A09696E74657276616C286DB9
:1004300073293A2025750A333A096D61785F737024
:100440006565643A2025750A343A0974696D655FFB
:10045000746F5F6D61783A2025750A353A097768BF
:1004600065656C5F6D61785F73706565643A2025C2
:10047000750A363A09776865656C5F74696D655F02
:10048000746F5F6D61783A2025750A00703A0970C3
:1004900072696E742076616C7565730A643A0973CB
:1004A00065742064656661756C74730A75703A09C9
:1004B0002B310A646E3A092D310A6C743A092B31DA
:1004C000300A72743A092D31300A4553432F713A7C
:1004D00009717569740A0A7370656564203D20644A
:1004E000656C7461202A206D61785F737065656446
:1004F000202A2028726570656174202F2074696D30
:10050000655F746F5F6D6178290A77686572652031
:1005100064656C74613A20637572736F723D256413
:100520002C20776865656C3D25640A5365652068F5
:100530007474703A2F2F656E2E77696B69706564DD
:1005400069612E6F72672F77696B692F4D6F7573B5
:10055000655F6B6579730A004D3E20004D25753A45
:1005600025733E20003F0A003D2025750A003F0A02
:100570000064656661756C74730A0025750A003F36
:100580000A000A092D2056616C756573202D0A003A
:10059000710A000A092D204D6F7573656B6579200E
:1005A0002D0A003F00433E20004C25640A000A0942
:1005B0002D20537461747573202D0A686F73745FF6
:1005C0006B6579626F6172645F6C65647328293A48
:1005D00020253032580A6B6579626F6172645F70F2
:1005E000726F746F636F6C3A20253032580A6B65F6
:1005F00079626F6172645F69646C653A202530329C
:10060000580A6B65796D61705F636F6E6669672EFE
:100610006E6B726F3A20253032580A74696D6572BC
:100620005F72656164333228293A202530386C586E
:100630000A000A092D2056657273696F6E202D0A13
:100640005649443A20307834383533284861737538
:1006500029205049443A20307839383043284643DD
:100660003938304329205645523A203078303130DD
:10067000300A4255494C443A2020284665622032CF
:10068000372032303232290A4F5054494F4E533AB4
:10069000204C554641204D4F5553454B455920451B
:1006A000585452414B455920434F4E534F4C4520CF
:1006B000434F4D4D414E44204E4B524F2034303924
:1006C000360A4743433A20352E342E3020415652C5
:1006D0002D4C4942433A20322E302E302041565282
:1006E0005F415243483A20617672350A000A092D6B
:1006F00020436F6E736F6C65202D0A4553432F7135
:100700003A09717569740A6D3A096D6F7573656B95
:1007100065790A000A092D204D61676963202D0A59
:10072000443A094465627567204D65737361676576
:1007300020546F67676C650A583A094D6174726995
:1007400078204465627567204D6F646520546F673B
:10075000676C65202D2053686F77206B6579707208
:10076000657373657320696E206D6174726978209A
:10077000677269640A4B3A094B6579626F6172640A
:1007800020446562756720546F67676C65202D2073
:1007900053686F77206B657970726573732072652B
:1007A000706F72740A4D3A094465627567204D6F27
:1007B00075736520546F67676C650A563A0956650C
:1007C0007273696F6E0A533A095374617475730AD0
:1007D000433A09416374697661746520436F6E73AF
:1007E0006F6C65204D6F64650A46312D4631303A95
:1007F0000953776974636820746F204C617965725E
:1008000020302D392028463130203D204C30290A17
:10081000302D393A0953776974636820746F204C1E
:100820006179657220302D390A47524156453A099F
:1008300053776974636820746F204C617965722006
:10084000302028616C7465726E617465290A423AC1
:10085000094A756D7020746F20426F6F746C6F6100
:100860006465720A4553433A094A756D7020746F86
:1008700020426F6F746C6F616465722028616C74C4
:1008800065726E617465290A453A095072696E7421
:1008900020454550524F4D2053657474696E6773FF
:1008A0000A4253504143453A09436C656172204501
:1008B0004550524F4D0A4E3A094E4B524F20546FFD
:1008C00067676C650A006B65796D61705F636F6E59
:1008D0006669672E7261773A20253032580A2E7386
:1008E0007761705F636F6E74726F6C5F636170735A
:1008F0006C6F636B3A2025750A2E636170736C6FA1
:10090000636B5F746F5F636F6E74726F6C3A2025F8
:10091000750A2E737761705F6C63746C5F6C6775BA
:10092000693A2025750A2E737761705F7263746C63
:100930005F726775693A2025750A2E737761705F5B
:100940006C616C745F6C6775693A2025750A2E734B
:100950007761705F72616C745F726775693A2025A8
:10096000750A2E6E6F5F6775693A2025750A2E73BA
:100970007761705F67726176655F6573633A2025A2
:10098000750A2E737761705F6261636B736C61735C
:10099000685F6261636B73706163653A2025750AF5
:1009A0002E6E6B726F3A2025750A0064656275675A
:1009B0005F636F6E6669672E7261773A2025303209
:1009C000580A2E656E61626C653A2025750A2E6D97
:1009D00061747269783A2025750A2E6B6579626FA9
:1009E0006172643A2025750A2E6D6F7573653A2021
:1009F00025750A006565636F6E6669673A0A646506
:100A00006661756C745F6C617965723A2025750A50
:100A1000003F004E4B524F3A206F66660A004E4B25
:100A2000524F3A206F6E0A000A6D6F7573653A2057
:100A30006F66660A000A6D6F7573653A206F6E0AFD
:100A4000000A6B6579626F6172643A206F66660AAC
:100A5000000A6B6579626F6172643A206F6E0A00FA
:100A60000A6D61747269783A206F66660A000A6DD1
:100A700061747269783A206F6E0A000A6465627563
:100A8000673A206F66660A000A64656275673A20F5
:100A90006F6E0A000A0A4A756D70696E6720746F7E
:100AA00020626F6F746C6F616465722E2E2E200051
:100AB000433E2000436C656172696E672045455076
:100AC000524F4D0A000A002530325820006B6579DC
:100AD000626F6172645F7265706F72743A20006455
:100AE000656C5F6B65795F6269743A2063616E273C
:100AF000742064656C3A20253032580A00616464C1
:100B00005F6B65795F6269743A2063616E27742058
:100B10006164643A20253032580A005B735D005BE3
:100B2000575D005B535D005B525D005B445D005BA5
:100B3000435D000E03460043003900380030004397
:100B40000000000A03480061007300750000000403
:100B500003090409025B00030100A0FA0904000074
:100B600001030101000921110100012240000705D4
:100B700081030800010904010001030000000921AC
:100B80001101000122B600070582032000010904BB
:100B900002000203000000092111010001222200CD
:100BA000070583032000010705030320000112014C
:100BB00000020000000853480C98000101020001E7
:100BC0000631FF0974A1010975150026FF00952063
:100BD000750881020976150026FF00952075089199
:100BE00002C005010902A10185020901A100050950
:100BF00019012908150025019508750181020501D3
:100C0000093009311581257F95027508810609385B
:100C10001581257F950175088106050C0A38021596
:100C200081257F950175088106C0C005010980A155
:100C300001850319012AB700150126B70095017532
:100C4000108100C0050C0901A101850419012AA029
:100C500002150126A002950175108100C005010949
:100C600006A1018506050719E029E715002501956C
:100C700008750181020507190029EF150025019566
:100C8000F075018102050819012905950575019185
:100C900002950175039101C005010906A10105072F
:100CA00019E029E7150025019508750181029501D4
:100CB000750881010507190029FF150026FF009519
:100CC000067508810005081901290595057501912A
:100CD00002950175039101C011241FBECFEFDAE028
:100CE000DEBFCDBF04B603FE18C0809169039091AA
:100CF0006A03A0916B03B0916C038730904BA740BF
:100D0000B04B59F41092690310926A0310926B036E
:100D100010926C03E0E0F8E3099511E0A0E0B1E087
:100D2000EEE5F6E502C005900D92A83EB107D9F7B1
:100D300023E0A8EEB1E001C01D92A936B207E1F7A9
:100D40000E9403180C942D2B0C940000FF93EF933A
:100D5000E091E801F091E901309709F00995EF91F0
:100D6000FF910895FC018591803011F0EFDFFBCFFA
:100D70000895FF27E0E230E247FF0CC0419597FF5E
:100D800009C0EDE26095709580959095611D711D8B
:100D9000811D911D27FF02C0219530E350E2AA2753
:100DA000660F771F881F991FAA1FA41710F0A41B96
:100DB00063955A95A9F7AA3008F0A95FA05DAF9393
:100DC000F395611571058105910541F7ED3211F437
:100DD000EF93F395F21718F43F93F395FBCF8F91B0
:100DE000B5DFFA95E1F70895E991F99185918030A1
:100DF00021F0853219F0AADFF9CF089520E0E894B8
:100E000055915532C1F3503311F4689455915A33CA
:100E100048F4505390F3220F022E220F220F200D80
:100E2000250FF4CF0EF4219589919991533619F33A
:100E3000533729F1533559F1BC0188279927E89494
:100E40005C3621F48991999168945591543639F41E
:100E500046EF7EF077FF0DC08FEF9FEF0AC055374A
:100E60004AE039F0583540E121F0523642E009F0CD
:100E70000895FF93EF937DDFEF91FF91B7CFFF933D
:100E8000EF93FC0181918030B9F360DFFBCFFF93DA
:100E9000EF9368DFF1CFDF93CF93CDB7DEB7259621
:100EA000A3DFCF91DF91089508950C9454070C941B
:100EB00054078091FE02816082608093FE0284B1BB
:100EC0008F6084B93E98469A3F9A8AB1806F8AB9FA
:100ED0005F9A479884B1806784B985B1806785B986
:100EE000EAEFF1E01192119282E0EA30F807D1F7CF
:100EF000EAEEF1E08AEF91E0119211928E179F07CE
:100F0000D9F78AEF91E090930D0280930C028AEE5C
:100F100091E090930B0280930A020C943709AF92F0
:100F2000BF92DF92EF92FF920F931F93CF93DF93C5
:100F300080910A0290910B0220910C0230910D02D7
:100F400030930B0220930A0290930D0280930C02BF
:100F5000C0E0D0E001E010E085B1807F8C2B85B946
:100F6000A8010C2E02C0440F551F0A94E2F7DA01C3
:100F7000A095B09520E030E08BB1682F6F78C90163
:100F800074E0880F991F7A95E1F7862B8BB99AE068
:100F90009A95F1F700C0C901880F991FE0910A02E4
:100FA000F0910B02E80FF91F6081718164237523B2
:100FB000672B09F0479AE5E3EA95F1F70000D6B40C
:100FC0005F98FAE0FA95F1F700C060910C02709119
:100FD0000D027B01E80EF91EF701369B05C0A080CB
:100FE000B180AA22BB2204C0A080B180A42AB52A65
:100FF000B182A082E6B5ED19E63068F0E0910A0210
:10100000F0910B02E80FF91FE080F180860F971F27
:10101000FC01F182E082FAE1FA95F1F700C047980D
:101020005F9A8BE291E00197F1F700C000002F5F1B
:101030003F4F2830310509F09FCFA0910C02B091AD
:101040000D02E0910A02F0910B0250962D913C9115
:101050005197808991892817390711F00E94A122A0
:101060002196C031D10509F077CF0E94390981E07E
:10107000DF91CF911F910F91FF90EF90DF90BF9084
:10108000AF90089520910C0290910D02E22FF92F5C
:10109000E80FF11DE80FF11D808191810895EF9215
:1010A000FF920F931F93CF93DF9385E691E00E9409
:1010B000B206C0E0D0E08EE7E82E81E0F82E06E52B
:1010C00011E08C2F0E9442080E94D609FF92EF92F5
:1010D0009F938F93DF93CF931F930F930E944B07A0
:1010E00021968DB79EB708960FB6F8949EBF0FBE97
:1010F0008DBFC830D10529F7DF91CF911F910F9196
:10110000FF90EF9008951F920F920FB60F92112447
:101110008F939F93EF93FF938091B900887F8038DE
:1011200069F038F48823C9F18036C9F510920E02AF
:1011300036C0883A09F1883BF9F031C080910E023F
:10114000811111C08091BB0080930F0280910F022A
:10115000803120F010920F0280E001C081E091E028
:1011600090930E021DC0E0910F02F0E08091BB0051
:10117000EA5BFC4F808308C0E0910F02F0E0EA5B7D
:10118000FC4F80818093BB0080910F0290E001961C
:101190008F70992780930F0202C01092BC0081E0EB
:1011A0009091BC008295880F880F807C9568892B70
:1011B0008093BC00FF91EF919F918F910F900FBE94
:1011C0000F901F9018950C94550781E0089581E0C9
:1011D00008950C94E70808950C94EB081F93CF939F
:1011E000DF9300D000D01F92CDB7DEB749835A837A
:1011F0006B833091110289819A81311114C0662369
:1012000059F0222349F00E949D0F182F682F8981E1
:101210009A810E94460F03C00E94710F182F6981A6
:101220007A81812F04C00E949D0F69817A810F907D
:101230000F900F900F900F90DF91CF911F910C9412
:10124000E116FC01262F40815181628173818481E6
:101250000C94EE0881E00895CF93DF93EC0160E0F9
:101260000E942109BE01DF91CF910C94EC080C94EF
:10127000E3080C94570708950E94F00D0E943B0963
:101280002FEF84E39CE0215080409040E1F700C0C4
:1012900000000C94E2220F931F93CF93DF938C01F5
:1012A00061E00E942109EC01B8010E94E90888234D
:1012B00009F45BC0B801CE010E942220882309F402
:1012C00054C0B801CE010E941B1B882309F44DC0F5
:1012D000B801CE010E947E1F882309F446C0F801A0
:1012E00082818823D9F1CF3D8CE5D80779F140F48C
:1012F000C115FCE5DF0791F0C130DC4591F02EC04F
:10130000CC35EDE5DE0741F1CD35FDE5DF0709F12F
:10131000CB35DD4519F50E94341420C00E943C09EC
:1013200024C08091FE02C82FC095C170C0FB80F917
:101330008093FE02CC2329F08DE893E00E94B20650
:1013400014C08BE793E00E94B20610C00E94E21422
:101350000CC00E942B1402C00E943714C801DF91F8
:10136000CF911F910F910C94E508C0E08C2FDF9175
:10137000CF911F910F9108950E9416220C94150A87
:101380000E94180A0C941C228295982F937344E0B3
:10139000949F900111248C7C86958695282B822F12
:1013A0008575880F2A7A2695822B0895CF93DF932F
:1013B000D92F0E94C409C82F8D2F0E94C4092C2F39
:1013C00030E0322F2227A901482BCA01DF91CF91AB
:1013D000089508950C94E90981E00895CF93C82FEA
:1013E0000E94EC09882379F0C0FF02C02C9A01C04A
:1013F0002C98C1FF02C02D9A01C02D98C2FF02C0D7
:101400002E9A01C02E98CF910895249A2C98259A4F
:101410002D98269A2E980895CF93C82F0E94EA09F6
:101420008C2F0E94EE09CF91089580E00C940C0A55
:101430000E947E200C940C0ACF930E947E20C82F1D
:1014400080911002C81741F1C09310028091FE02F2
:1014500082FF1EC080FF04C085EA93E00E94B206AE
:101460008091FE0280FF0CC01F92CF9380EA93E030
:101470009F938F930E944B070F900F900F900F90A8
:101480008091FE0280FF04C08EE993E00E94B206C4
:101490008C2FCF910C940C0ACF910895CF93DF93AA
:1014A000CDB7DEB72B970FB6F894DEBF0FBECDBF1A
:1014B0004F83588769877A878B8761110E946313EE
:1014C0009E012F5F3F4F86E0F90111928A95E9F75F
:1014D00085E0FE013796D90101900D928A95E1F7DA
:1014E00089819A814C815D81452B31F09F3F31F498
:1014F00091E08F3F19F403C091E001C090E090FFAC
:1015000009C049815A816B817C818D819E810E94B5
:10151000841205C0C9010E942A098111F2CF2B96BD
:101520000FB6F894DEBF0FBECDBFDF91CF91089507
:10153000FC01808191810E94DF0F0895CF93882361
:1015400009F455C0C82F8CEF8C0F813AF8F48C2F1A
:101550000E94271F81114BC06C2F80910201909136
:1015600003010E942F21882349F06C2F80910201F2
:10157000909103010E94DC210E9485136C2F8091C1
:101580000201909103010E94D1210CC080E28C0FD6
:10159000883058F4C77081E001C0880FCA95EAF717
:1015A0000E944613CF910C948513EBE5EC0FE330CA
:1015B00040F4F0E0E95BFE4F808190E0CF910C9425
:1015C000ED20E8E5EC0FE73150F4F0E0EE0FFF1FFF
:1015D000E75EFE4F80819181CF910C940321CD3E37
:1015E00030F08C2F0E948818CF910C945A19CF910B
:1015F0000895882389F19CEF980F913A40F4682F61
:1016000080910201909103010E94DC210DC090E2C3
:10161000980F983058F4877091E001C0990F8A951F
:10162000EAF7892F0E944C130C9485139BE5980FC1
:10163000933020F480E090E00C94ED2098E5980F32
:10164000973120F480E090E00C9403218D3E20F04F
:101650000E94E3180C945A1908951F93CF93DF93B7
:10166000182FEB010E949E0A209741F08FE99FE01E
:101670000197F1F700C000002197F6CF812FDF918D
:10168000CF911F910C94F90A893319F060E070E052
:1016900002C060E570E00C942D0B882321F00E94BD
:1016A00046130C9485130895882321F00E944C134F
:1016B0000C9485130895CF92DF92EF92FF920F93CF
:1016C0001F93CF93DF937C01D62FC72FFC0112818C
:1016D000058102950F700E943C138823B9F01123F5
:1016E000A9F08C2F807F803421F080E28D0F88302C
:1016F00068F08091570382FD09C082E00E94E513E3
:101700000E943C1391E0D82ED92601C0D12CCC2EBA
:10171000C2948FE0C8228C2D90E08C30910508F0A7
:10172000CFC1FC01EA5AFF4F0C94C42A8C2F807F52
:10173000CF70882311F0C295C07F112399F0CC237C
:1017400009F4AAC180E28D0F883010F0D11104C0D5
:101750008C2F0E94461303C08C2F0E9456130E94A8
:1017600085139AC18D2F0E94F90ACC2309F4A8C1D0
:1017700080E28D0F883038F1DD2329F18C2F0E9413
:101780005C1324C08C2F807FCF70803211F0C29503
:10179000C07FDD2319F0D130A1F13DC08091570306
:1017A00082FF17C0112349F0CC2329F08C2F0E940F
:1017B00046130E94851380E070C180E00E94F90A00
:1017C000CC2309F47DC18C2F0E944C130E948513F9
:1017D00077C1112371F0002341F0013031F40E94F0
:1017E00066138C2B0E946E136BC10E9466138C2BA8
:1017F0001DC0002319F0013009F462C10E947B135F
:1018000025C0112321F0063008F05AC10EC0053062
:1018100008F056C11BC0112361F0002331F0F7011D
:10182000858180FF39C18F7085838C2F0E944D0B7D
:1018300047C1002359F0D93309F03FC1FFEF07EE4C
:1018400013E0F15000401040E1F735C18C2F0E94A9
:10185000540B36C18C2F86958695837019F0813094
:1018600061F02EC1112321F08D2F9C2F937002C0A7
:1018700080E090E00E94ED202BC1112321F08D2FFC
:101880009C2F937002C080E090E00E94032120C151
:101890008D2F112319F00E94881802C00E94E318AE
:1018A0000E945A1915C18C2F837009F047C011117D
:1018B0000BC12D2F229526952770220F220F6D2FF9
:1018C0006F70862F90E0A0E0B0E0022E04C0880F79
:1018D000991FAA1FBB1F0A94D2F7D4FF10C04FE074
:1018E00050E060E070E004C0440F551F661F771F92
:1018F0002A95D2F7409550956095709503C040E0C9
:1019000050E0BA01C695C695C3708A019B01082BA9
:10191000192B2A2B3B2BC901B801C23049F058F4CE
:10192000C13019F00E945C0ECFC00E944A0ECCC09C
:101930000E946E0EC9C00E94480EC6C0112319F045
:101940008C2F817001C08695882309F4BDC02D2F8E
:10195000229526952770220F220F6D2F6F70862FEC
:1019600090E0A0E0B0E0022E04C0880F991FAA1FEB
:10197000BB1F0A94D2F7D4FF10C04FE050E060E0E4
:1019800070E004C0440F551F661F771F2A95D2F7D9
:10199000409550956095709503C040E050E0BA01C5
:1019A000C695C695C3708A019B01082B192B2A2B5B
:1019B0003B2BC901B801C23049F058F4C13019F0CD
:1019C0000E94210F81C00E940F0F7EC00E94330F22
:1019D0007BC00E94820E78C0CF70112339F08C2F0B
:1019E0000E94A80E8D2F0E944D0B6EC08D2F0E945D
:1019F000540B8C2F0E94C90E67C0D23F21F128F4EE
:101A0000D03F41F0D13FC1F043C0D33F19F1D43FA3
:101A100079F03EC0112341F0053008F051C08C2F01
:101A20008F710E94EE0E4CC0063008F049C0F7CF0F
:101A30008091570382FF18C0112339F08C2F8F71CA
:101A40000E94A80E3DC01123C9F38C2F8F710E94F4
:101A5000C90E36C0112329F08C2F8F710E94930E6E
:101A60002FC00E948E0E2CC0112349F0CF718C2FF5
:101A70000E94A80E63E08C2F0E94CA1321C081E04F
:101A80000E94E5130230E0F082E00E94E51318C0E6
:101A9000112331F0002391F28D2F0E949E0A10C075
:101AA000002399F2D93349F41FEF27EE33E01150A8
:101AB00020403040E1F700C000008D2F0E94F90A5D
:101AC00088EF8C0D843020F40E947E200E940C0A46
:101AD000DD20C9F00E94381380FD15C0F701128285
:101AE0000E9432130E94A80EC7010E94A40D0E94FA
:101AF0003213DF91CF911F910F91FF90EF90DF9004
:101B0000CF900C94C90EDF91CF911F910F91FF9050
:101B1000EF90DF90CF9008950F931F93CF93DF93B3
:101B2000EC01688179818A810E94EA0F8C010E9410
:101B3000450F0E94360EB801CE010E945B0BDF916B
:101B4000CF911F910F910895CF93DF93EC0198816E
:101B500089812B813C81232B31F08F3F31F481E04F
:101B60009F3F19F403C081E001C080E080FD1DC0EB
:101B7000CE010E944B09811110C00E943C138823A2
:101B8000A1F08A81882389F08091570382FD0DC0DE
:101B900082E0DF91CF910C94E513CE010E948C0D71
:101BA000CE01DF91CF910C942C09DF91CF91089554
:101BB00080E090E00E94ED2080E090E00E94032110
:101BC0000E9463130E9485130E940D1B0C945A19E6
:101BD00080910201909103010E94E7210C94D80D9D
:101BE0000E9453130C94E80D92959F70963079F0F3
:101BF00010F4925001C09A50923068F4803F69F01E
:101C000018F4883E40F409C0843F29F406C0883E99
:101C100020F0813F11F080E0089581E00895FC01FB
:101C2000808191810E94DF0F0E94F40D0895CF936F
:101C3000DF9300D000D01F92CDB7DEB70F900F908A
:101C40000F900F900F90DF91CF910895CF93DF9376
:101C500000D000D000D0CDB7DEB726960FB6F894EE
:101C6000DEBF0FBECDBFDF91CF91089508950895D7
:101C70000C94370E0C94380E0E943A0E6093660254
:101C80007093670280936802909369020C94D80D58
:101C90000C943C0E0F931F93009166021091670203
:101CA0002091680230916902602B712B822B932B5B
:101CB0001F910F910C943C0E0F931F93009166029D
:101CC00010916702209168023091690260237123AC
:101CD000822393231F910F910C943C0E0F931F931B
:101CE00000916602109167022091680230916902AA
:101CF00060277127822793271F910F910C943C0E28
:101D00000C94370E0E94800E6093620270936302FF
:101D100080936402909365020C94D80D60E070E0AB
:101D2000CB010C94820E0F931F9341E050E060E0D2
:101D300070E08A019B0104C0000F111F221F331F96
:101D40008A95D2F7C901B8011F910F910C94820EA8
:101D50000F931F9341E050E060E070E004C0440F37
:101D6000551F661F771F8A95D2F780916202909166
:101D70006302A0916402B09165028A019B01082B65
:101D8000192B2A2B3B2BC901B8011F910F910C94E1
:101D9000820E0F931F9341E050E060E070E004C0BA
:101DA000440F551F661F771F8A95D2F740955095AF
:101DB000609570958091620290916302A091640297
:101DC000B09165028A019B01082319232A233B2332
:101DD000C901B8011F910F910C94820E0F931F93AC
:101DE00041E050E060E070E004C0440F551F661F02
:101DF000771F8A95D2F78091620290916302A09139
:101E00006402B09165028A019B01082719272A27DD
:101E10003B27C901B8011F910F910C94820E0F93BB
:101E20001F9300916202109163022091640230912D
:101E30006502602B712B822B932B1F910F910C94B9
:101E4000820E0F931F930091620210916302209102
:101E500064023091650260237123822393231F91D2
:101E60000F910C94820E0F931F93009162021091B8
:101E700063022091640230916502602771278227F6
:101E800093271F910F910C94820E089520E1929F49
:101E9000800D1124E82FE695E695E695877051E0D0
:101EA00001C0550F8A95EAF785E0E89FF0011124FB
:101EB000EE5EFD4F20E030E070E04081CB01022E6D
:101EC00002C0969587950A94E2F7817081958427E0
:101ED0008523842781932F5F3F4F2530310569F794
:101EE000089520E1929F800D1124682F66956695D4
:101EF0006695982F977085E0689FB001112440E0A7
:101F000050E080E0FB01E40FF51FEE5EFD4F208105
:101F100030E0092E02C0369527950A94E2F7217029
:101F20003327042E01C0220F0A94EAF7822B4F5F59
:101F30005F4F4530510531F70895BF92CF92DF9240
:101F4000EF92FF920F931F93CF93DF938C01C0907A
:101F50006202D0906302E0906402F090650280918A
:101F6000660290916702A0916802B0916902C82A46
:101F7000D92AEA2AFB2ACFE1D0E0D701C6010C2EEC
:101F800004C0B695A795979587950A94D2F780FDDA
:101F900004C0219790F7B12C07C0BC2EB8018C2F3C
:101FA0000E94F6160197A9F38B2DDF91CF911F9117
:101FB0000F91FF90EF90DF90CF90BF900895CF9357
:101FC000DF93EC010E949D0FBE010E94F616DF9187
:101FD000CF9108951F93CF93DF93EB01909111025E
:101FE000992321F0CB010E94DF0F13C0882349F011
:101FF000CB010E949D0F182F682FCE010E94460F23
:1020000004C0CB010E94710F182FBE01812F0E94C6
:10201000F616DF91CF911F9108951F93CF93DF9311
:10202000C0916A0216E080916B02C81799F0D0E067
:102030001C9FF0011D9FF00D1124E459FD4F4081BC
:10204000518162817381848195810E94260E21963F
:10205000C770E9CFDF91CF911F91089540919C0205
:1020600050919D0260919E0270919F028091A0020A
:102070009091A1020C94260EEF92FF920F931F9362
:10208000CF93DF938091A10282958F7009F065C094
:1020900080919E02882309F460C080916A02F090CA
:1020A0006B0210919C0200919D0260919F027091C1
:1020B000A00291E01F3F09F090E0C0910001D09193
:1020C0000101292F96E0E92E8F1509F446C061150C
:1020D000710521F00F3F21F030E003C031E001C075
:1020E000322F90E030FD36C0E89EF001E99EF00D01
:1020F0001124DF01A459BD4F11963C911197301363
:1021000029C03C91311326C012963C91129731118F
:1021100021C013964D915C911497461B570B4C1799
:102120005D07C0F48091A1028F7080618093A1024D
:10213000EF58FD4F80818F70806180838CE992E041
:102140000E94A40DDF91CF911F910F91FF90EF900E
:102150000C940D1001968770B7CFDF91CF911F912E
:102160000F91FF90EF9008959F92AF92BF92CF9200
:10217000DF92EF92FF920F931F93CF93DF93CDB730
:10218000DEB761970FB6F894DEBF0FBECDBF8C01EE
:1021900085E0F801DE011D9601900D928A95E1F728
:1021A000D8011296EC9090919C02E0919D022091B2
:1021B0009F023091A0022115310531F0EF3F31F43B
:1021C00081E09F3F19F403C081E001C080E0B82F97
:1021D000B1709B2E80FD47C1D8014C9111965C9146
:1021E00011971396AD90BC9014978CE9C82E82E09D
:1021F000D82EF0909E02B501621B730B2091000156
:1022000030910101FF2009F4D9C08091A102621729
:10221000730708F095C0282F207F09F052C05E1385
:1022200013C0491311C0FE2CE1100EC08F708061E5
:102230008093A1020E942E10C6010E94A40D8091DD
:10224000A102F80185834DC1AB2831F05F3F31F425
:1022500081E04F3F19F403C081E001C080E080FDC0
:1022600003C081E08E2502C080E090E0F82FF1707D
:10227000FF2E80FF1CC080916A0220916B0236E025
:10228000821709F40BC190E0389FF001399FF00DDF
:102290001124E459FD4F6181561306C06081461335
:1022A00003C06281E61203C001968770E9CFFE2C5D
:1022B000EE2009F416C18091A10281608093A102F1
:1022C00054C05E1306C0491304C0E11002C0F801F7
:1022D00099C0C8010E940F0E882361F1EE2051F1D0
:1022E0002091A102822F82958F7090E0029774F066
:1022F00080919C0290919D0298878F831986BB865E
:10230000AA862C87CE0107960E94A40D86E0F801CC
:10231000ACE9B2E001900D928A95E1F70E943C1081
:102320000E942E100AC05E1711F1C8010E940F0E04
:1023300081112CC0C8010E94A40DFF24F394D1C0C8
:10234000282F207F81F77A2DB98AA88A6E2D898956
:102350000E94170E8CE992E00E94A40D86E0D6013F
:102360001D928A95E9F70E942E10F12CBAC04913EC
:10237000DCCFE110DACFF8018583C8010E94A40DFB
:1023800086E0D6011D928A95E9F7ABC0EE2091F266
:102390002091A102822F82958F7090E002970CF419
:1023A000B5CF80919C0290919D029A8389831B8274
:1023B000BD82AC822E83CE010196A6CF6217730731
:1023C00008F044C0FE2CEE2009F4B4CF5E1330C0F8
:1023D00049132EC02091A10220FD21C0822F829599
:1023E0008F70482F50E041155105C9F0F801258341
:1023F0004F30510541F08F5F982F9295907F822F3B
:102400008F70892B8583C8010E94A40D86E0F80196
:10241000ACE9B2E001900D928A95E1F73CC086E00C
:10242000F801ACE9B2E001900D928A95E1F759C04C
:10243000C8010E940F0E811169CF8091A1028160B5
:102440008093A102C8010E94A40D4BC07A2DB98AC5
:10245000A88A6E2D89890E94170E86E0D6011D92EA
:102460008A95E9F718C0EE2009F464CFC8010E94EC
:102470000F0EF82E882309F45DCF86E0F801ACE951
:10248000B2E001900D928A95E1F78CE992E00E940A
:10249000980A0E943C100E942E1023C04D875E8730
:1024A0008D859E850E94DF0F292F22952F70223067
:1024B00028F49F7039F0811105C00BC0243028F436
:1024C0009F7049F4805E883020F0C8010E94A40DFE
:1024D0009F2CF92C06C0D80115969C91907F91F7FE
:1024E000F8CF8F2D61960FB6F894DEBF0FBECDBF2B
:1024F000DF91CF911F910F91FF90EF90DF90CF90E0
:10250000BF90AF909F9008951F93CF93DF93CDB767
:10251000DEB72C970FB6F894DEBF0FBECDBF4F834A
:10252000588769877A878B879C87CE0107960E9498
:10253000B4108823D1F09F8188852A853B85232B81
:1025400031F08F3F31F481E09F3F19F403C081E007
:1025500001C080E080FD47C04F81588569857A853C
:102560008B859C850E94260E3EC086E0FE01379634
:10257000DE01119601900D928A95E1F7FF81E885C1
:102580006A857B856115710531F0EF3F31F481E09B
:10259000FF3F19F403C081E001C080E080FD23C04B
:1025A00020916B0230E0C901019687709927409114
:1025B0006A0250E084179507F1F1F983EA837D837D
:1025C0006C8396E0929FD001939FB00D1124A45983
:1025D000BD4FFE01319601900D929A95E1F78093DF
:1025E0006B020E940D1016E080916A0290916B02BE
:1025F000891771F1189FC001112484599D4F0E94C1
:10260000B410882329F1E0916A021E9FF001112481
:10261000E459FD4F408151816281738184819581AC
:102620000E94260E80916A0290E001968770992799
:1026300080936A02D9CF0E94F00D10926B02109223
:102640006A02ECE9F2E086E0DF011D928A95E9F783
:102650002C960FB6F894DEBF0FBECDBFDF91CF91A1
:102660001F9108958091C20285958595859508955D
:102670008091C202877008959091C202977081E0A4
:1026800009F480E008958091E50208959091E502B3
:10269000892B8093E502089580959091E502892326
:1026A0008093E50208951092E50208959091E40266
:1026B000892B8093E402089580959091E402892308
:1026C0008093E40208951092E40208958091C30279
:1026D000089508950C9469130C946A13909157030C
:1026E00092FD08C09091C302981721F08093C30215
:1026F0000C946C1308958091C302882329F01092E2
:10270000C30280E00C946C130895CF93DF93E091A3
:102710000201F09103018091E5028083E0910201C2
:10272000F091030190818091E402892B8083809154
:10273000C302882381F0E0910201F09103019081AE
:10274000892B808380910201909103010E941921BD
:1027500081110E947B13C0910201D091030140E2DC
:1027600050E062EA72E0CE010E94DE2A892B69F015
:1027700080E2FE01A2EAB2E001900D928A95E1F7B3
:10278000CE01DF91CF910C948A20DF91CF910895F3
:102790000C9469139091570392FD10C098E0899FA3
:1027A00090011124262B2093C2020E94A80E809132
:1027B000C2028595859585950C94C8130C94A80E36
:1027C0001092C20280E00C94C8132091C20280953E
:1027D00082238093C202982F977099F430E0482F9B
:1027E000082E000C550B2417350759F0909157030C
:1027F00092FD07C08595859585950E94C90E0C941C
:10280000E0130895CF939091570392FB222720F96C
:102810002817F9F0C82F892FC0FB82F9809357033E
:1028200080915603909157030E945E1482E00E94AB
:10283000E5138091FE0280FF0CC01F92CF9380EBC6
:1028400093E09F938F930E944B070F900F900F90F0
:102850000F90CF9108958091570382FB882780F9CC
:1028600091E089270C94021481E00C94021480E01A
:102870000C94021480E090E00E94F32A21E0893E4B
:102880009E4F09F020E0822F089582E090E00C94A2
:10289000EB2A83E090E00C94EB2ACF9384E090E065
:1028A0000E94EB2AC82F82E290E00E94EB2A2C2F94
:1028B00030E0A901582BCA01CF910895CF93C92FB9
:1028C000682F84E090E00E94F92A6C2F82E290E069
:1028D000CF910C94F92AAB01BC018FE090E00C94ED
:1028E0000B2BAB01BC0183E190E00C940B2B60E05F
:1028F00070E0CB010C94711460E070E0CB010E9499
:102900006B140C94771469EE7EEF80E090E00E94E7
:10291000172B60E082E090E00E94F92A60E083E0FB
:1029200090E00E94F92A10926602109267021092BB
:1029300068021092690260E084E090E00E94F92A47
:1029400060E082E290E00E94F92A60E085E090E099
:102950000E94F92A60E086E090E00E94F92A6FEF79
:1029600087E090E00E94F92A40E050E0BA0188E058
:1029700090E00E940B2B60E08DE090E00E94F92A2D
:1029800040E050E0BA0188E190E00E940B2B60E04B
:1029900087E190E00E94F92A40E050E0BA018CE122
:1029A00090E00E940B2B60E070E080E290E00E94DB
:1029B000172B40E050E0BA0188E190E00E940B2B19
:1029C0000C947C140C948314682F8EE090E00C948B
:1029D000F92A0E94A1226093FA027093FB0280936D
:1029E000FC029093FD026093F6027093F7028093CD
:1029F000F8029093F902089585B7806885BF85B77E
:102A0000806885BF089581E008950C9403150895AA
:102A10000C9407150C9407150C940A150C940715C3
:102A20000C940E150C9407150E94FC148EEE94E283
:102A30000E9474200E9412150C9410150E94081513
:102A40000C9407150E94D3170C94050A0E948C223F
:102A50000E9459070E9422150C940C155F926F92E8
:102A60007F928F929F92AF92BF92CF92DF92EF921E
:102A7000FF920F931F93CF93DF93CDB7DEB72A97C3
:102A80000FB6F894DEBF0FBECDBF0E948F07C82ED1
:102A900081110E94E91436EE832E32E0932E00E07D
:102AA00010E0502E802F0E9442085C01F4016190DA
:102AB00071904F016826792661147104B1F40F5F9B
:102AC0001F4F0830110569F78FEF89838A831B82B6
:102AD0000E9495228160782F9D838C8349815A8141
:102AE0006B818D810E944E0A3AC08091FE0281FD69
:102AF0000E944F08D12CEE24E394F12CC3018E21C7
:102B00009F21892B29F10E9405158823A9F0DE82D7
:102B10005F82AE20BF2081E0AB2809F480E0888787
:102B20000E9495228160782F9A8789874E815F81E4
:102B300068858A850E944E0A000F111FF801EA512C
:102B4000FD4F80819181E826F926F182E08207C05D
:102B5000D394EE0CFF1CF0E1DF12D0CFB0CF81E0B8
:102B6000C11001C080E02A960FB6F894DEBF0FBEF8
:102B7000CDBFDF91CF911F910F91FF90EF90DF902C
:102B8000CF90BF90AF909F908F907F906F905F900D
:102B900008950E942E150E94FA190C941C0ACF93D6
:102BA000DF930E94FB16EC01811521E5920708F0E6
:102BB00045C0811530E5930708F094C0883E910523
:102BC00028F5803E910508F0F8C0883A910570F428
:102BD000853A910508F07CC08130910509F475C0F3
:102BE00008F4E8C0049708F0E8C0E4C08F3B910502
:102BF00008F0E0C0C85AD0E0CC0FDD1FC65BDE4F46
:102C00000990D881C02DCE019464D8C0811540E2CE
:102C1000940758F4811551E0950708F0CEC08D3E19
:102C2000910508F4C7C09065C9C0C11580E4D807F4
:102C300008F4C0C0DF70CE01906AC0C0811525E5E0
:102C40009207A8F4811534E5930708F095C0811523
:102C500043E5940708F07BC0811552E5950708F01D
:102C600061C0D82FCC27CE01816F906AA7C0C11553
:102C700089E5D807A0F4C11528E5D20708F082C07D
:102C8000C11536E5D30708F095C08C2F0E948F1729
:102C90008F7190E0D82FCC27CE0190628FC0C115E4
:102CA0004AE5D40708F474C0CE01905681159042CD
:102CB00008F080C08D2F8F710E948F17DD27D062A2
:102CC0008F71AE01582BCA0179C081E090E076C0C7
:102CD000C55AD0E0C858DE4F8881C82FD0E0CE0159
:102CE00090646CC074E0969587957A95E1F7282FEB
:102CF00023703C2F337081E090E002C0880F991F51
:102D00003A95E2F79C68AC01522B9A019C2F9F7078
:102D10009695969550E2959FE0011124C9018C2B60
:102D20009D2B4CC08370992721E030E002C0220F18
:102D3000331F8A95E2F79C2F9695969580E2989F8F
:102D4000E0011124C22BD32BCE019C6837C08370C5
:102D5000992721E030E002C0220F331F8A95E2F765
:102D60009C2F9695969540E2949FE0011124C22BEA
:102D7000D32BCE019A6822C0D82FCC27CE01846FE6
:102D8000906A1CC0DC2FCC27CE01806F906A16C0E1
:102D90008C2F8F700E948F1794E0D695C7959A95C7
:102DA000E1F7CF70D0E0DC2FCC27D0699E01282B33
:102DB000C90104C080E090E001C0CE01DF91CF9155
:102DC0000895E72FF0E098E0899FE00DF11D1124B0
:102DD00084E0EE0FFF1F8A95E1F7E60FF11DEE0F7D
:102DE000FF1FE558FE4F8591949108950E94E116CA
:102DF0000E94CF1508958238910569F1B0F48133AE
:102E0000910509F46DC048F48932910509F463C055
:102E10008A32910509F469C008958533910509F452
:102E200055C089339105B9F00895833E910569F144
:102E300038F4803E9105B1F0823E910509F1089584
:102E4000863E9105A9F1873E9105B9F1843E910531
:102E500009F064C023C02091560320FD4FC021FD1E
:102E60004DC008958091560380FD44C08091570362
:102E700080FF44C08091560384FD42C083EE4DC064
:102E80008091560382FF38C0F5CF8091560382FDB2
:102E900033C08091570380FD31C0ECCF8091570340
:102EA00081FF32C08091560384FD2AC087EE35C071
:102EB0008091560383FF26C0F5CF8091560383FD92
:102EC00021C08091570381FD1FC0ECCF8091560334
:102ED00085FD1CC01DC08091560385FD19C016C01C
:102EE0008091560386FD16C017C08091560386FD5B
:102EF00013C010C089E311C082EE0FC080EE0DC078
:102F000080E00BC086EE09C084EE07C089E205C0F0
:102F100085E303C08AE201C081E390E008959091C7
:102F2000560392FF0DC0282F2871283019F4877F8F
:102F3000846006C0282F2471243011F48B7F8860B0
:102F400093FF0DC0282F2871283119F4877E8461E2
:102F500006C0282F2471243111F48B7E88612091C2
:102F6000570320FF0DC0382F3871383019F4877F90
:102F7000816006C0382F3171313011F48E7F886046
:102F800021FF0DC0282F2871283119F4877E816117
:102F900006C0282F2171213111F48E7E886194FDA5
:102FA000877E089508950E943A14811102C00E94FC
:102FB000E2140E9445148093FE020E944D149093E7
:102FC0005703809356030E94D2170E944914682F1A
:102FD00070E080E090E00E94480E60916202709183
:102FE000630280916402909165020C94800E0E94AD
:102FF0006A250E9426150C9476250E947A250E9447
:10300000C9150C9498250E9433220E9451250E94D4
:1030100014150E94F7170E94FD170E941E15FBCF82
:103020008091050380FF06C06091090170E0660F82
:10303000771F26C081FF04C06091090184E005C0AC
:1030400082FF07C06091090188E0689FB0011124E8
:1030500017C0909104039923D1F06091080196174D
:1030600088F72091090188E0289F90011124929F00
:10307000A001939F500D112470E0CA010E94B02A54
:103080006038710540F46115710519F406C068E0F7
:1030900070E0862F08958FE7089581E0089580916C
:1030A000050380FF08C06091050170E07595679584
:1030B0007595679521C081FF06C06091050170E09C
:1030C0007595679519C082FF04C06091050170E095
:1030D00010C090910303992399F060910401961711
:1030E000A0F780910501899FC001112470E00E9422
:1030F000B02A6038710540F46115710519F406C0F5
:1031000061E070E0862F08958FE7089581E00895CB
:103110008D3E21F40E941018819504C08E3E29F442
:103120000E9410188093090308958F3E21F40E9495
:103130001018819504C0803F29F40E9410188093D4
:1031400008030895893F19F40E944F1805C08A3F6B
:1031500031F40E944F18819580930A0308958B3FA4
:1031600021F40E944F18819504C08C3F29F40E94DD
:103170004F1880930B0308959FE0980F983078F4D0
:1031800021E030E0A90102C0440F551F9A95E2F7F3
:10319000CA0190910703892B8093070308958D3FFF
:1031A00021F48091050381600BC08E3F21F4809152
:1031B0000503826005C08F3F29F480910503846078
:1031C0008093050308958D3E39F49091090397FF8C
:1031D00035C01092090359C08E3E29F4909109031D
:1031E0001916BCF32BC0909108038F3E29F497FF6A
:1031F00025C01092080349C0803F19F41916CCF37A
:103200001DC090910A03893F29F41916BCF410924D
:103210000A033BC08A3F19F497FF10C0F8CF8B3FD9
:1032200039F490910B0397FF09C010920B032DC046
:103230008C3F21F490910B031916BCF39FE0980F7B
:10324000983080F421E030E0A90102C0440F551FFE
:103250009A95E2F7CA01809590910703892380939C
:10326000070313C08D3F21F4809105038E7F0BC0AF
:103270008E3F21F4809105038D7F05C08F3F29F497
:10328000809105038B7F8093050380910803811152
:1032900006C080910903811102C01092040380913D
:1032A0000A03811106C080910B03811102C01092A4
:1032B000030308958091FE0283FF7EC08CEE93E0AD
:1032C0000E94B206809107031F928F9387EE93E0CE
:1032D0009F938F930E944B0785EE93E00E94B20666
:1032E00080910803282F082E000C330B3F938F93F7
:1032F00082EE93E09F938F930E944B0780EE93E0C2
:103300000E94B20680910903282F082E000C330B6F
:103310003F938F938DED93E09F938F930E944B0784
:103320008BED93E00E94B20680910A03282F082EAD
:10333000000C330B3F938F9388ED93E09F938F9313
:103340000E944B0786ED93E00E94B20680910B032A
:10335000282F082E000C330B3F938F9383ED93E0BF
:103360009F938F930E944B0780ED93E00E94B206DB
:10337000809104031F928F938DEC93E09F938F9322
:103380000E944B078BEC93E00E94B20680910503EC
:103390001F928F9388EC93E09F938F930E944B072B
:1033A00085EC93E00E94B2068DB79EB74C960FB69F
:1033B000F8949EBF0FBE8DBF0E94952220910803F6
:1033C000211104C020910903222321F090930203CC
:1033D0008093010320910A03211104C020910B0363
:1033E000222321F0909300038093FF0286E093E074
:1033F0000C94DF20EF92FF920F931F93CF93DF93F4
:1034000000D000D000D0CDB7DEB786E0E6E0F3E034
:10341000DE01119601900D928A95E1F7E090080384
:10342000F090090300910A0310910B031092080316
:103430001092090310920A0310920B03E11003C0CB
:10344000FF2009F45DC080910103909102030E9466
:10345000AD22AC0190910403992339F020910A0127
:1034600030E02417350758F04BC020910B018AE05B
:10347000289F900111242417350718F041C09F3F61
:1034800019F09F5F90930403EE2061F00E941018E2
:103490001E1414F09FEF01C091E0989F902D11240D
:1034A00090930803FF2061F00E9410181F1414F07D
:1034B0009FEF01C091E0989F902D112490930903F4
:1034C000309108033323E1F0209109032223C1F056
:1034D00045EB3403C0011124992319F0909308039C
:1034E00003C081E08093080335EB2303C00111245E
:1034F000992319F09093090303C081E08093090395
:10350000011103C0112309F45DC08091FF02909165
:1035100000030E94AD22AC0190910303992339F07E
:103520002091060130E02417350758F04BC0209158
:1035300007018AE0289F900111242417350718F00D
:1035400041C09F3F19F09F5F90930303002361F0F8
:103550000E944F18101614F09FEF01C091E0989F41
:10356000902D112490930A03112361F00E944F18AB
:10357000111614F09FEF01C091E0989F902D112437
:1035800090930B0330910A033323E1F020910B0356
:103590002223C1F045EB3403C0011124992319F013
:1035A00090930A0303C081E080930A0335EB230361
:1035B000C0011124992319F090930B0303C081E0FB
:1035C00080930B038091080381110BC08091090344
:1035D000811107C080910A03811103C080910B0300
:1035E00081110E945A19EB82FC820D831E8386E0B2
:1035F000FE013196A6E0B3E001900D928A95E1F7C5
:1036000026960FB6F894DEBF0FBECDBFDF91CF91E7
:103610001F910F91FF90EF900895E6E0F3E086E0B0
:10362000DF011D928A95E9F71092040310920303BB
:10363000109205030895CF93DF93EC01FB01828183
:10364000882309F43CC1C430FDE5DF0760F4CB3FBB
:103650009CE5D90788F49E0122503C452431310570
:1036600008F02EC109C0C236EDE5DE0729F0C63AE2
:10367000FDE5DF0709F024C10E944D149093570324
:1036800080935603C1318CE5D80709F4C6C008F011
:1036900042C0C930ECE5DE0709F49BC000F5C53037
:1036A0008CE5D80709F485C078F4C330ECE5DE0773
:1036B00009F478C008F07AC0C230DC4509F0F5C0E2
:1036C000809156038160EFC0C7309CE5D90709F4AB
:1036D00078C008F07AC0809156038061E4C0CD3094
:1036E000FCE5DF0709F487C058F4CB309CE5D90727
:1036F00009F479C008F07BC08091560388606FC0E0
:10370000CF30FCE5DF0709F480C008F082C080916B
:103710005603877FC8C0CE3F9CE5D90709F471C026
:1037200000F5C531FCE5DF0709F485C068F4C33155
:103730009CE5D90709F475C008F095C00E94F00D0A
:10374000809156038F77AFC0CC3FFCE5DF07A9F12E
:1037500008F054C0CB3FDC4509F0A7C08091570367
:1037600040C0C230EDE5DE0709F489C058F4C11548
:103770008DE5D80709F45AC008F069C08091570355
:1037800082602FC0C236EDE5DE0709F47CC0C63A80
:10379000FDE5DF0709F481C0C330DD4509F085C0D0
:1037A00080E06EC08091560382607DC08091560398
:1037B00016C080915603886076C08091570382605E
:1037C0004FC08091560380626EC080915603806422
:1037D0006AC00E94F00D80915603806864C08460C6
:1037E00062C081603DC0809156038E7F5CC0809135
:1037F00056038D7F58C08091560316C080915703A1
:1038000018C0809157038D7F2BC0809156038F7E07
:103810004AC0809156038F7D46C0809156038F7BAE
:1038200042C080915603877F8B7F3DC080915703B4
:103830008D7F8E7F15C08091560382FB222720F951
:1038400091E0922790FB82F990FB83F92CC0809144
:103850005703982F909591708E7F892B90FB81F95B
:103860008093570322C00E94F00D8091560387FB7E
:10387000222720F991E0922790FB87F914C081E07C
:103880000E94E41412C08091560384FB222720F981
:1038900091E0922790FB84F906C080915603982FFF
:1038A000909590FB80F980935603809156039091F8
:1038B00057030E945E140E94F00D80E001C081E079
:1038C000DF91CF910895809104011F928F93809191
:1038D00005011F928F93809108011F928F93809111
:1038E00009011F928F9380910A011F928F938091FB
:1038F0000B011F928F938FE094E09F938F930E9410
:103900004B078DB79EB70E960FB6F8949EBF0FBEAD
:103910008DBF0895883220F58E3108F068C08B3055
:1039200091F1C0F4873009F0BEC081E080930B01B3
:1039300084E180930A018AE0809309018EE18093FB
:10394000080188E08093050188E28093040181E703
:1039500095E0C6C0833109F443C0843169F1A3C046
:103960008F3409F49EC028F4893231F1883359F03C
:103970009AC0813531F008F4D4C0823509F4A7C06B
:1039800092C08FEFA5C083E995E00E94B2060E9425
:10399000631C1F9281E08F931F9288E08F938CE8C5
:1039A00094E09F938F930E944B070F900F900F907E
:1039B0000F900F900F9096C080E995E00E94B2069C
:1039C00080911003882309F4AAC01092100310926A
:1039D0000F0310920E0310920D0310920C03B1C04E
:1039E00082E895E00E94B2060E94631C7BC08D5164
:1039F00080931003833031F170F48130D1F0823044
:103A000009F03FC08AE091E090930F0380930E038A
:103A100088E891E01FC0853059F108F1863089F5BA
:103A200084E091E090930F0380930E0383EC91E088
:103A300011C08BE091E090930F0380930E038FE70A
:103A400091E008C089E091E090930F0380930E030A
:103A500084E991E090930D0380930C0318C088E0F3
:103A600091E090930F0380930E0381EA91E0F2CFEF
:103A700085E091E090930F0380930E0380EB91E03B
:103A8000E9CF109210038FE795E00E94B206809173
:103A90001003882309F455C01F928F938BE795E09C
:103AA0000DC08AE015C08EE695E01AC097FF47C0AA
:103AB000108280811F928F9388E695E09F938F9369
:103AC0000E944B070F900F900F900F900BC081E05A
:103AD000E0910E03F0910F03309729F585E695E00C
:103AE0000E94B20620911003222359F180910C0309
:103AF00090910D03009711F48BE791E09F938F93C2
:103B00001F922F938CE595E09F938F930E944B0714
:103B10000F900F900F900F900F900F9016C080E0B5
:103B2000089586EFD5CF2081082E000C990B820FC7
:103B3000911D8F3F910509F00CF4B8CF8FEF808372
:103B4000B8CF88E595E00E94B20681E00895CF9352
:103B5000C82F1F928F9389EA95E09F938F930E94BD
:103B60004B0781E090E0A0E0B0E0BC01CD0104C0D3
:103B7000660F771F881F991FCA95D2F70E94480EBB
:103B80000F900F900F900F90CF910C94F00DDF924B
:103B9000EF92FF920F931F93CF93DF93482F50E044
:103BA000FA013597EF33F10508F03FC1EE59FF4FA9
:103BB0000C94C42A0E9449141F928F9384EF99E0B9
:103BC0009F938F930E944B070E94451483FB992774
:103BD00090F91F929F9382FB992790F91F929F93D0
:103BE00081FB992790F91F929F93982F91701F92B4
:103BF0009F931F928F938BEA99E09F938F930E94DC
:103C00004B070E944D1487FB222720F91F922F9308
:103C100086FB222720F91F922F9385FB222720F96C
:103C20001F922F9384FB222720F91F922F9383FB4F
:103C3000222720F91F922F9382FB222720F91F921F
:103C40002F9391FB222720F91F922F93292F217068
:103C50001F922F9381FB222720F91F922F93282F49
:103C600021701F922F939F938F9386EC98E09F93E0
:103C70008F930E944B078DB79EB788960FB6F89426
:103C80009EBF0FBE8DBF06C084EB9AE00E94B206B5
:103C90000E94E214C1E0CEC084E197E074C080913C
:103CA000FE02817F8E7F8093FE028DEE96E00E9461
:103CB000B20680EB9AE00E94B20681E08093110385
:103CC000E9CF84E99AE00E94B2060E943C09E2CF63
:103CD0008091FE02C82FC095C170C0FB80F980930F
:103CE000FE02CC2319F088E89AE091C08BE79AE0B5
:103CF0000E94B2068091FE02897F877F8093FE0238
:103D0000C9CF9091FE0291FBCC27C0F981E0C82772
:103D1000892FC0FB81F98093FE02CC2319F08EE637
:103D20009AE027C080E69AE02EC09091FE0292FBB6
:103D3000CC27C0F981E0C827892FC0FB82F9809386
:103D4000FE02CC2319F081E59AE013C081E49AE0E9
:103D50001AC09091FE0293FBCC27C0F981E0C827DE
:103D6000892FC0FB83F98093FE02CC2351F085E3B9
:103D70009AE00E94B2068091FE0281608093FE026A
:103D800059C088E29AE00E94B20684CF82E396E0AE
:103D9000FACF0E94A122062FF72EE82ED92EC0912D
:103DA0005603C7FBCC27C0F910914503D0911801E9
:103DB0000E947E20DF92EF92FF920F931F92CF938B
:103DC0001F921F931F92DF931F928F938EEA95E0AD
:103DD0009F938F930E944B078DB79EB70E960FB699
:103DE000F8949EBF0FBE8DBF55CF0E94F00D9091ED
:103DF000560397FBCC27C0F981E0C827892FC0FB69
:103E000087F980935603CC2329F08EE19AE00E9433
:103E1000B20610C083E19AE0B6CF895303C08D513A
:103E200001C080E00E94A71D35CF81E19AE00E9489
:103E3000B206C0E08C2FDF91CF911F910F91FF90C0
:103E4000EF90DF90089580E008950C94231FCF93A6
:103E5000C82F80911103813071F040F0823009F059
:103E600045C08C2F0E948A1C81E046C00E944313EB
:103E70008232F1F504C00E944313823261F48C2F28
:103E80000E94251F811104C08C2F0E94C71D2CC0C9
:103E900081E090E029C08C2F0E94231F811123C054
:103EA000C431C9F058F4CB3069F0C031B9F482E0C4
:103EB0008093110388E30E948A1C15C0C93259F00F
:103EC000C83361F48DEE96E00E94B20685EA95E073
:103ED0000E94B20608C0109211030CC083EA95E05C
:103EE0000E94B20607C081E0817006C010921103E3
:103EF00080E002C080E0F8CFCF910895CF93DF93A8
:103F000086319C4541F5EB010E944313982F8A812D
:103F10002091020130910301882379F09A7A81E09F
:103F200009F480E080931203911102C069E201C09C
:103F300065E3C9010E94D1210AC080911203811159
:103F400002C069E201C065E3C9010E94DC210E9450
:103F5000851380E001C081E0DF91CF9108950F9338
:103F60001F93CF93DF93C42FD22FFC01828188232C
:103F7000C9F0409315030E949522909314038093F7
:103F8000130380E28C0F883008F057C0C77081E0BF
:103F900001C0880FCA95EAF7DF91CF911F910F9169
:103FA0000C944D0B80911503481330C0809113037E
:103FB000909114030E94AD22883C910538F510E2DF
:103FC0001D0FCD17B9F080E28C0F883040F4C77018
:103FD00081E001C0880FCA95EAF70E94540B18309F
:103FE00028F581E09D2F977001C0880F9A95EAF718
:103FF0000E944D0B802F0E94440B1830F0F4D770B4
:1040000081E001C0880FDA95EAF70AC080E28C0FE0
:10401000883098F4C77081E001C0880FCA95EAF72C
:10402000DF91CF911F910F910C94540B802FDF9152
:10403000CF911F910F910C94440BDF91CF911F9161
:104040000F9108950F939C01CB01243F4CE5340759
:1040500031F188F4293DFCE53F07D9F02A3D4CE5D4
:10406000340779F1283D3C45A9F506E221EE41EE01
:1040700068ED7CE52BC0263FFCE53F07E1F0A8F0AA
:10408000273F3C4539F507E225EE46EE67EF7CE534
:104090001DC007E225EE45EE69ED7CE517C006E29E
:1040A00021EE40EE64EF7CE511C007E225EE44EE20
:1040B00065EF7CE50BC006E221EE42EE66EF7CE5A3
:1040C00005C008E221E045EE6AED7CE50E94AF1FE5
:1040D00080E008C0FC018281882319F0109215034A
:1040E00001C081E00F9108959093E9018093E80168
:1040F000089590931B0380931A030895E0911A0387
:10410000F0911B03309721F00190F081E02D09948C
:1041100080E00895EF92FF921F93CF93DF93FC010D
:10412000A0911A03B0911B03109709F442C080912B
:104130001801882341F08091560387FF04C08081D5
:10414000818386E08083EF011296ED91FC911397B5
:10415000CE0109958091FE0282FF2BC080FF04C032
:104160008DEC9AE00E94B20618E087ECE82E8AE017
:10417000F82E8091FE0280FF0BC088811F928F93E2
:10418000FF92EF920E944B070F900F900F900F90AD
:10419000115021961111EDCF8091FE0280FF09C0D0
:1041A00085EC9AE0DF91CF911F91FF90EF900C94F6
:1041B000B206DF91CF911F91FF90EF900895E091AB
:1041C0001A03F0911B03309739F022E0DC012C93A5
:1041D0000480F581E02D0994089520911803309111
:1041E00019032817390771F0909319038093180366
:1041F000E0911A03F0911B03309721F00680F781BC
:10420000E02D099408952091160330911703281783
:10421000390771F09093170380931603E0911A0306
:10422000F0911B03309721F00084F185E02D099473
:104230000895FC01329680911801882331F0809115
:10424000560387FF02C09EE101C096E080E09150D6
:1042500028F021912223D9F38F5FF9CF08956623A7
:1042600051F1209118012223E9F02091560327FFF4
:1042700019C0462F4695469546954E31E0F4677035
:1042800021E030E002C0220F331F6A95E2F7FC0103
:10429000E40FF11D828190E02823392381E0232B54
:1042A00069F409C0FC01329608962191621729F041
:1042B000E817F907D1F780E0089581E008959C019F
:1042C000FC0132969FEF80E04191461789F09F3FB5
:1042D00019F4411101C0982F8F5F8630A9F79F3FD5
:1042E00039F0F901E90FF11D97FDFA956283089500
:1042F00008959C012A5F3F4FFC014281461301C093
:104300001282019682179307B9F70895262F2695F2
:10431000269526952E3170F4FC01E20FF11D677091
:1043200021E030E001C0220F6A95EAF78281282B54
:10433000228308958091FE0280FF0CC01F926F932C
:104340008DEF9AE09F938F930E944B070F900F90F1
:104350000F900F900895262F2695269526952E319D
:1043600078F4FC01E20FF11D677021E030E001C03C
:10437000220F6A95EAF720958281282322830895E7
:104380008091FE0280FF0CC01F926F938FED9AE028
:104390009F938F930E944B070F900F900F900F9059
:1043A000089520911801222329F02091560327FD1A
:1043B0000C9486210C945F2120911801222329F06E
:1043C0002091560327FD0C94AB210C947921209168
:1043D0001801FC013296222331F08091560387FFA9
:1043E00002C08EE101C086E0DF011D928A95E9F7E7
:1043F000089508950C94F92183E080931C030C9494
:10440000FA21811102C081E001C082E080931C0387
:104410000C94FA210C94012281E080931C030C94EB
:10442000FA210C940C2208950C9413220C9414225B
:104430000C9413220C9413220C941322CF930E94F9
:104440001A220E948F070E941822C0E08C2F0E941F
:104450004208892B29F4CF5FC830C1F780E001C042
:1044600081E0CF91089508951F920F920FB60F9299
:1044700011248F939F93AF93BF9380911D0381115C
:1044800013C08091580390915903A0915A03B091A1
:104490005B034196A11DB11D80935803909359036E
:1044A000A0935A03B0935B03BF91AF919F918F91FB
:1044B0000F900FBE0F901F9018958091600384306D
:1044C00031F10E94BC0910921D0320E488E190E0C4
:1044D0000FB6F894A895809360000FBE20936000FB
:1044E00083B7817F846083BF83B7816083BF789403
:1044F000889583B78E7F83BF0FB6F894A895809177
:104500006000886180936000109260000FBE089583
:104510000E94F00D0C94C00982E084BD93E095BD2B
:104520009AEF97BD80936E0008952FB7F89480910D
:10453000580390915903A0915A03B0915B032FBF88
:1045400008952FB7F89460915803709159038091A2
:104550005A0390915B032FBF08959C014FB7F894C5
:104560008091580390915903A0915A03B0915B0335
:104570004FBF821B930B089578941F920F920FB632
:104580000F9211248F939F93AF93BF938091580301
:1045900090915903A0915A03B0915B030196A11D1C
:1045A000B11D8093580390935903A0935A03B0937D
:1045B0005B03BF91AF919F918F910F900FBE0F90B2
:1045C0001F90189581E08093E00080E28093D800EE
:1045D0001092C9008FE19EE40197F1F700C000003E
:1045E00087E090EBDC018093690390936A03A093CA
:1045F0006B03B0936C039CE088E10FB6F894A89528
:10460000809360000FBE90936000FFCF80914403C1
:104610000895089522E02093E9002FEF3091E800FB
:10462000215035FD06C035ED3A95F1F70000211116
:10463000F5CF2091E80025FF0BC040E050E066E098
:1046400070E00E9407268091E8008E778093E80052
:104650000895CF93DF9320911801222339F0209100
:10466000560327FF03C060E222E002C068E021E0B9
:104670002093E9002FEF3091E800215035FD06C06E
:1046800035ED3A95F1F700002111F5CF2091E800C2
:1046900025FF1DC0EC0180911801811105C040E08B
:1046A00050E068E070E003C070E040E050E0CE0110
:1046B0000E9407268091E8008E778093E80080E2D0
:1046C000FE01A4E2B3E001900D928A95E1F7DF913B
:1046D000CF91089580932003709322036093210368
:1046E00080916003843001F582E08093E9008FEFD0
:1046F0009091E800815095FD06C095ED9A95F1F7EF
:1047000000008111F5CF8091E80085FF0DC040E0E9
:1047100050E063E070E080E293E00E940726809121
:10472000E8008E778093E8000895BC0184E00C9443
:104730006A23BC0183E00C946A238FE29BE00E9411
:10474000B20680915F03811109C00E9498270E94E0
:10475000F5278091E20084608093E20008958BE267
:104760009BE00E94B20610925F03089587E29BE0EF
:104770000E94B2060C94112283E29BE00E94B206D2
:1047800060915C0381E0611101C080E00C94FC2128
:104790008FE19BE00E94B2069091600381E094302B
:1047A00009F080E060915C030C94012220911F03CA
:1047B0002F5F822F62E30E94A42A992319F020938D
:1047C0001F03089510921F0380912303882371F122
:1047D00080916003843041F58091E9008F702091D1
:1047E000EC00922F917020FD90E8892B93E090933C
:1047F000E9009091EB0090FF14C09091EE0097FFBC
:1048000010C09091E80095FF03C01092F100F9CF1D
:104810009091E80090FF05C09091E8009E779093FA
:10482000E8008F708093E90010922303089542E01E
:1048300061EC81E00E94112742E261EC82E00E947B
:10484000112742E261EC83E00E94112790916003FE
:1048500081E0943009F080E060915C030C940A22BE
:1048600080916203833009F461C030F4813071F0CB
:10487000823009F49AC008958A3009F486C08B30DA
:1048800009F46CC0893009F0A8C020C08091610390
:10489000813A09F0A2C08091E800877F8093E80008
:1048A0008091650390916603892B21F460E284E294
:1048B00093E003C060E080E090E070E00E94522648
:1048C0008091E8008B778093E800089580916103E0
:1048D000813209F082C0809165039091660302974E
:1048E00008F07BC08091E800877F8093E80080918A
:1048F000E80082FD05C0809160038111F8CF6DC092
:104900002091F3008091F20090E0922B029731F415
:104910008091F100813011F0863021F48091F10016
:10492000809344038091E8008B7753C080916103AA
:10493000813A09F052C08091650390916603892BFA
:1049400009F04BC08091E800877F8093E800809158
:10495000E80080FFFCCF8091180136C08091610390
:104960008132D9F58091650390916603892BA9F571
:104970008091E800877F8093E8000E94462780911D
:104980006303809318010C94F00D809161038132D0
:1049900021F58091E800877F8093E8000E944627F8
:1049A0008091640380934503089580916103813A67
:1049B000A1F48091E800877F8093E8008091E8006F
:1049C00080FFFCCF809145038093F1008091E80047
:1049D0008E778093E8000C94462708959FB7F8944B
:1049E000109223039FBF90916003943009F057C049
:1049F0009091E9009F703091EC00232F217030FDE1
:104A000020E8922B23E02093E9002091EB0020FF87
:104A100043C02091EE0027FF3FC020911E032223B8
:104A200021F02091E80025FF37C010921E0326E0F8
:104A30003091E80035FD15C030916003343061F5E8
:104A40003091EB0035FD28C0215021F481E08093A6
:104A50001E0322C0EFE9FFE03197F1F700C000002C
:104A6000E7CF8093F1008091E80085FD0AC0809136
:104A7000E80080FFFCCF8091E8008E778093E8000B
:104A800006C08FB7F89421E0209323038FBF9F7057
:104A90009093E90080E008959F709093E9008FEF74
:104AA000089584B7877F84BF0FB6F894A895809146
:104AB0006000886180936000109260000FBE90E0FB
:104AC00080E80FB6F89480936100909361000FBE68
:104AD0000C940C220E9498270E94F527E2EEF0E049
:104AE00080818460808378940C94892A8CE091E0A2
:104AF0000C947920809160038530C9F48BE19BE0B0
:104B00000E94B20680916003853079F40E945D2294
:104B100080915E038823B1F30E941E22882391F3C3
:104B20000E94F1250E94F00DEDCF0C94882208958B
:104B300008950C949B25292F332723303105C9F084
:104B400060F42130310581F02230310509F041C097
:104B50008BE590E023E53BE040C021323105E1F0F8
:104B60002232310531F135C082E190E02EEA3BE09E
:104B700034C099278130910549F028F0029749F512
:104B8000E3E3FBE005C0EFE4FBE002C0E3E4FBE0AD
:104B9000849190E09F0121C063307105D0F4660FCD
:104BA000771FFB01EF51FE4F2081318189E090E0BA
:104BB00014C06330710568F4FB01EE0FFF1FE5526E
:104BC000FE4F20813181FB01E852FE4F808190E051
:104BD00004C080E090E020E030E0FA0131832083DF
:104BE000089580E189BD82E189BD09B400FEFDCF51
:104BF0008091D8008F7D8093D8008091E000826002
:104C00008093E0008091E00081FDFCCF0895CF9279
:104C1000DF92EF92FF920F931F93CF93DF93EC01FC
:104C20008B017A010E946527811133C0E114F104E0
:104C300039F0F70180819181081B190BC80FD91F2A
:104C4000C12CD12C0115110519F18091E80085FDC9
:104C500016C08091E8008E778093E800E114F1049B
:104C600049F0F70180819181C80ED91ED182C0829E
:104C700085E00FC00E946527882321F30AC089912F
:104C80008093F10001501109FFEFCF1ADF0ADACF4C
:104C900080E0DF91CF911F910F91FF90EF90DF9017
:104CA000CF90089520916703309168032617370746
:104CB00048F06115710539F42091E8002E772093B2
:104CC000E80001C0B901FC0120E06115710579F12E
:104CD000809160038823F1F18530F1F18091E80043
:104CE00083FD3CC08091E80082FD2EC08091E800E9
:104CF00080FFEBCF2091F3008091F20090E0922BA7
:104D00006115710551F08830910538F42191209397
:104D1000F100615071090196F3CF21E0089709F085
:104D200020E08091E8008E778093E800CECF2111BB
:104D3000CFCF0AC080916003882361F0853061F095
:104D40008091E80083FD0AC08091E80082FFF2CFE5
:104D500080E0089582E0089583E0089581E0089559
:104D600020916703309168032617370748F06115D3
:104D7000710539F42091E8002E772093E80001C0F6
:104D8000B901FC0120E06115710591F1809160038A
:104D9000882309F440C0853009F43FC08091E800C1
:104DA00083FD3DC08091E80082FD2FC08091E80026
:104DB00080FFE9CF2091F3008091F20090E0922BE8
:104DC0006115710559F08830910540F424912093C4
:104DD000F1003196615071090196F2CF21E00897F8
:104DE00009F020E08091E8008E778093E800CBCF37
:104DF0002111CCCF0AC080916003882361F08530F7
:104E000061F08091E80083FD0AC08091E80082FF94
:104E1000F2CF80E0089582E0089583E0089581E074
:104E20000895982F973068F59093E900981739F016
:104E30007091EC002091ED005091F00003C0242F00
:104E4000762F50E021FD02C09F5FECCF3091EB0048
:104E50003E7F3093EB003091ED003D7F3093ED00CD
:104E60003091EB0031603093EB007093EC002093B5
:104E7000ED005093F0002091EE0027FDE5CF80E09B
:104E800008958F708093E90081E008958091610317
:104E900087FF11C08091E80082FD05C0809160030A
:104EA0008111F8CF11C08091E8008B770BC0809101
:104EB0006003882349F08091E80080FFF8CF80915B
:104EC000E8008E778093E80008952091E400309107
:104ED000E50095E64091EC00842F817040FF23C0EF
:104EE0008091E80080FD1DC080916003882399F0C7
:104EF000853099F08091EB0085FD11C04091E40070
:104F00005091E5002417350729F3915011F09A01CB
:104F1000E1CF84E0089582E0089583E0089581E080
:104F2000089580E008954091E80042FFDDCF0895A4
:104F30000E9406280E940E28E0EEF0E08081816049
:104F40008083E8EDF0E080818F77808319BCA7ED46
:104F5000B0E08C918E7F8C9380818F7E80831092C5
:104F60005F0308950F931F93CF93DF930E9406284A
:104F70000E940E28C8EDD0E088818F7788838881D1
:104F80008068888388818F7D888319BC1092600334
:104F900010925C0310925E0310925D0300EE10E02D
:104FA000F80180818B7F808388818160888342E0E3
:104FB00060E080E00E941127E1EEF0E080818E7FCA
:104FC0008083E2EEF0E08081816080838081886070
:104FD0008083F80180818E7F8083888180618883CF
:104FE000DF91CF911F910F910895E8EDF0E080815E
:104FF0008F7E8083E7EDF0E080818160808384E0B4
:1050000082BF81E080935F030C94B227E8EDF0E06B
:1050100080818E7F80831092E20008951092DA00E2
:105020001092E10008951F920F920FB60F92112473
:105030002F933F934F935F936F937F938F939F93A0
:10504000AF93BF93EF93FF938091E10082FF0BC07A
:105050008091E20082FF07C08091E1008B7F809306
:10506000E1000E94D6238091DA0080FF1FC080916A
:10507000D80080FF1BC08091DA008E7F8093DA0019
:105080008091D90080FF0DC080E189BD82E189BD9A
:1050900009B400FEFDCF81E0809360030E949D2350
:1050A00005C019BC109260030E94AF238091E100FB
:1050B00080FF19C08091E20080FF15C08091E2005E
:1050C0008E7F8093E2008091E20080618093E20015
:1050D0008091D80080628093D80019BC85E08093CD
:1050E00060030E94BC238091E10084FF30C0809166
:1050F000E20084FF2CC080E189BD82E189BD09B452
:1051000000FEFDCF8091D8008F7D8093D8008091E4
:10511000E1008F7E8093E1008091E2008F7E80939A
:10512000E2008091E20081608093E20080915C0364
:10513000882311F084E007C08091E30087FD02C05E
:1051400081E001C083E0809360030E94C8238091C6
:10515000E10083FF29C08091E20083FF25C0809198
:10516000E100877F8093E10082E0809360031092EA
:105170005C038091E1008E7F8093E1008091E200EA
:105180008E7F8093E2008091E20080618093E20054
:1051900042E060E080E00E9411278091F00088608A
:1051A0008093F0000E94B623FF91EF91BF91AF91E1
:1051B0009F918F917F916F915F914F913F912F912F
:1051C0000F900FBE0F901F9018951F920F920FB661
:1051D0000F9211242F933F934F935F936F937F937D
:1051E0008F939F93AF93BF93CF93DF93EF93FF93EF
:1051F000C091E900CF708091EC00D82FD17080FD74
:10520000D0E81092E9008091F000877F8093F00051
:1052100078940E9429291092E9008091F00088601A
:105220008093F000CD2BCF70C093E900FF91EF91F8
:10523000DF91CF91BF91AF919F918F917F916F91AE
:105240005F914F913F912F910F900FBE0F901F9044
:1052500018951F93CF93DF93CDB7DEB7AA970FB6FC
:10526000F894DEBF0FBECDBFE1E6F3E08091F10020
:10527000819323E0E936F207C9F70E943024809138
:10528000E80083FF2EC18091610390916203492F52
:1052900050E04A30510508F024C1FA01EF55FF4FA4
:1052A0000C94C42A803821F0823809F01AC108C051
:1052B00080915D0390915E03992389F082600FC015
:1052C000809165038F70873008F00BC18093E900EF
:1052D0008091EB0085FB882780F91092E90090917E
:1052E000E800977F9093E8008093F1001092F1001E
:1052F000D1C0282F2D7F09F0F4C0882319F0823007
:1053000061F0EFC080916303813009F0EAC093300F
:1053100009F080E080935E032EC0809163038111C9
:105320002AC0809165038F702FEF280F263008F078
:10533000D8C08093E9002091EB0020FF1CC093307F
:1053400021F48091EB00806214C09091EB00906199
:105350009093EB0021E030E0A90102C0440F551FFB
:105360008A95E2F74093EA001092EA008091EB0000
:1053700088608093EB001092E9008091E800877FBD
:105380008093E8000E944627ACC08111AAC010910A
:1053900063031F778091E3008078812B8093E30083
:1053A0008091E800877F8093E8000E9446278091E3
:1053B000E80080FFFCCF8091E30080688093E300E9
:1053C000111102C082E001C083E08093600389C0B4
:1053D0008058823008F085C0809163039091640307
:1053E0008C3D53E0950779F583E08A838AE28983CF
:1053F0004FB7F894DE01139620E03EE051E2E32F30
:10540000F0E050935700E49120FF03C0E295EF7065
:105410003F5FEF708E2F90E0EA3010F0C79601C02A
:10542000C0968D939D932F5F243149F74FBF809194
:10543000E800877F8093E8006AE270E0CE01019681
:105440000E94522616C06091650370916603AE01FA
:105450004F5F5F4F0E949925BC01892B09F441C021
:105460009091E800977F9093E80089819A810E944B
:10547000B0268091E8008B778093E80032C08038B6
:1054800081F58091E800877F8093E80080915C033C
:105490008093F1008091E8008E7772CF811121C056
:1054A000809163039091640399270297D4F48091CB
:1054B000E800877F8093E8008091630380935C031A
:1054C0000E94462780915C03811106C08091E30011
:1054D00087FD02C081E001C084E0809360030E94E8
:1054E00017248091E80083FF0AC08091E800877F3D
:1054F0008093E8008091EB0080628093EB00AA9695
:105500000FB6F894DEBF0FBECDBFDF91CF911F91D4
:105510000895CF93809160038823A1F0C091E900A2
:10552000CF709091EC00892F817090FD80E8C82B9E
:105530001092E9008091E80083FD0E942929CF7034
:10554000C093E900CF910895991B79E004C0991F99
:10555000961708F0961B881F7A95C9F780950895CD
:1055600097FB072E16F4009407D077FD09D00E9410
:10557000CA2A07FC05D03EF4909581959F4F089567
:10558000709561957F4F0895EE0FFF1F0590F49180
:10559000E02D0994AA1BBB1B51E107C0AA1FBB1F2A
:1055A000A617B70710F0A61BB70B881F991F5A95AF
:1055B000A9F780959095BC01CD010895FB01DC0110
:1055C00004C08D910190801921F441505040C8F7DA
:1055D000881B990B0895F999FECF92BD81BDF89A69
:1055E000992780B50895A8E1B0E042E050E00C941E
:1055F0001F2B262FF999FECF92BD81BDF89A0197F6
:1056000000B4021639F01FBA20BD0FB6F894FA9A0A
:10561000F99A0FBE08950396272F0E94FA2A0E9436
:10562000F92A252F0E94FA2A242F0C94FA2A01968F
:10563000272F0E94FA2A0C94F92ADC01CB01FC01E5
:10564000F999FECF06C0F2BDE1BDF89A319600B4DB
:0E5650000D9241505040B8F70895F894FFCFE6
:10565E00C800C402280850011E0A1401062329237B
:10566E000A2399239523092301E200E900EA00B5F4
:10567E0000B600B700CD008301CC008A01920194E0
:10568E00012102230224022502260227022A02B346
:10569E0000B4006F007000818283E200E900EA002E
:1056AE00B500B600B700CD008301CC008A0192018F
:1056BE0094012102230224022502260227022A0235
:1056CE00B300B4006F0070008182833F3F3F006DD6
:1056DE006B5F64656C6179006D6B5F696E7465728A
:1056EE0076616C006D6B5F6D61785F73706565647C
:1056FE00006D6B5F74696D655F746F5F6D617800CF
:10570E006D6B5F776865656C5F6D61785F737065F3
:10571E006564006D6B5F776865656C5F74696D6558
:10572E005F746F5F6D61780040B622980CE20BC01B
:08573E000B650B7E0B970B00BD
:00000001FF
